:10000000280F0020B9320000B5320000B5320000E0
:1000100000000000000000000000000000000000E0
:10002000000000000000000000000000B5320000E9
:100030000000000000000000B5320000B5320000F2
:10004000B5320000B53200008D1C0000B532000052
:1000500095160000B5320000B5320000352C0000C6
:10006000B5320000B5320000B5320000B5320000F4
:10007000B5320000B5320000B5320000B5320000E4
:10008000B5320000B5320000B5320000B5320000D4
:10009000B5320000B5320000B5320000B5320000C4
:1000A000B5320000B5320000B5320000B5320000B4
:1000B00008B5064B064803331B1A062B00D808BDAB
:1000C000044B002BFBD09847F9E7C04604370000EB
:1000D000043700000000000008B50748074B1B1A52
:1000E0009B10DA0FD318591000D108BD044A002A1A
:1000F000FBD09047F9E7C046043700000437000002
:100100000000000010B5074C2378002B09D1FFF741
:10011000CFFF054B002B02D0044800E000BF0123B5
:10012000237010BD640100200000000004370000AF
:1001300008B5094B002B03D00848094900E000BF6F
:1001400008480368002B03D0074B002B00D09847CA
:10015000FFF7C2FF08BDC0460000000004370000E2
:1001600068010020043700000000000010B572B6DE
:10017000BFF35F8F194A002313701948D9B20133B6
:100180001818013800780028F7D0002905D101237C
:100190001370BFF35F8F62B61FE072B6BFF35F8F5D
:1001A000002313704B1EDBB2022B07D9032B0CD19B
:1001B0000C4B042019690143196106E00949042424
:1001C0000869A043086108494B7001231370BFF30D
:1001D0005F8F62B6BFF34F8F30BF10BD5801002054
:1001E0009404002000ED00E00004004013B5184B1B
:1001F0001A68110603D41968FD220A401A7001F02A
:10020000A5F8144C144A80231B05062163600820BE
:100210001170A36101F0B4F8226A6B461201D20F8B
:10022000DA7107331B78002B03D10C4B9B6B9A06BA
:100230000CD58022D2011368591C00D1FEE783F34C
:100240000888074B9A60074B1B68984713BDC04648
:1002500000100040004400415B44004100040040A5
:1002600000ED00E00440000013B5FFF7BFFF184B9E
:1002700001221A70BFF35F8F62B6164B00241A7109
:100280001C705C709C70DC7001F0F5FC6A46124BCF
:10029000147054705B686846DB061B0F9370D47053
:1002A000147101F083F80D4B802252059A6100F021
:1002B00039F800F03FF800F013FE094B1B78002BD3
:1002C00003D000F0EDFC0028F7D1FFF74FFFF4E773
:1002D00058010020940400200040004100440041E7
:1002E0008001002008B500F025F808BD08B500F031
:1002F00029F808BD08B5044B1B78002B03D001F08A
:1003000095FF00F02BF808BD80010020014B012073
:100310001870704780010020014B00221A7070474E
:1003200080010020024B802252059A617047C0462E
:1003300000440041024B802252055A617047C0467A
:1003400000440041024B802252059A617047C0462A
:10035000004400417047704770477047002804D13F
:100360008022064B52059A6107E0FA239B009842CF
:1003700003D18022014B52055A617047004400416D
:10038000024B1878431E98414000704781010020BD
:10039000054B1A780223002A03D1E423FF330360BC
:1003A000131C181C7047C0468101002000207047B4
:1003B00001207047F22370B55B00051C0E1C012064
:1003C0009D4217D84A1900249A4213D8A0B2B042CD
:1003D0000FD2401980B200F0AFF880220120064908
:1003E0009200002300F0A0FC01340028EED101208F
:1003F00000E0002070BDC04694020020F8B5F22352
:10040000051C0E1C5B0001209D4216D84A190024D1
:100410009A4212D8A7B20020B7420ED280220749D2
:100420009200031C00F080FC002805D07F19B8B2B0
:1004300000F06EF80134EDE70120F8BD94020020D1
:1004400043081B1810B5DBB2094AC40708D5D45CB1
:100450000F2020400C012043D0540909D31805E097
:100460000F20D154D3180A0A81431143597010BD8B
:1004700094020020F7B5224B00915A335D781A7828
:100480002D021543013DAD00ADB2A84237D3E022A5
:10049000FF32AB189BB2984231D8451BE0236D0266
:1004A0005B00EB1801932C1C8022009BD201A61844
:1004B000144F002B06D07F1B3919301C402201F04D
:1004C00045F80BE0F3B2002B02D1301C01F076F8B6
:1004D0007F1B3919301C402200F0EEFF019A403496
:1004E0009442E1D1084B009AE8180849002A03D049
:1004F000402201F02BF802E0402200F0DDFFF7BDC2
:100500000000002094020020C0410000540400209C
:1005100008B502280AD9032805D1054960220548F3
:1005200003F004F802E00021FFF7A4FF08BDC04675
:10053000940200200000002038B5234C8022051CC6
:100540000021201C920003F033F8281E032836D81F
:1005500002F0E4FE020F0F2F3E22201C1B4902F086
:10056000E5FFFF2355225B00E254194BAA22E25417
:1005700028E000201749FFF763FF01201649FFF725
:100580005FFF164B00245A335D781A782D0215430D
:10059000A3B25819E2B280B2772A03D0691C591865
:1005A00089B200E00C490134FFF74AFF782CEFD103
:1005B00008E0201C0949602202F0B8FF02E0012196
:1005C000FFF758FF38BDC046940200206C3600008B
:1005D000FF010000F80F0000FF0F000000000020E6
:1005E00073B501AC01250026211C1C206570A67086
:1005F000257001F06DF8054B802252055A611B20D1
:10060000211C2670657001F063F873BD0044004141
:100610000120704708B5031C0120002B01D1FFF712
:10062000AFFE08BD021C08B50120002A02D1081C3B
:10063000FFF7AEFE08BD031C0020834201D101205C
:100640004840704708B5031C0120002B01D1FFF77B
:10065000ADFE08BD08B5031C0120002B01D1FFF73A
:10066000A7FE08BD002801D1014800E00020704726
:10067000AA360000F8B5071C0E1C151C0124FFF754
:1006800069FE002F04D1301C291CFFF793FE041CC7
:10069000FFF761FE201CF8BDF8B5071C0E1C151CE9
:1006A0000124FFF759FE002F04D1301C291CFFF74D
:1006B000A5FE041CFFF751FE201CF8BD002070476A
:1006C000431E9841034BC0B21870034B01221A70AD
:1006D0007047C046990400206000002010B5054C0A
:1006E0000021201C122202F063FFF02323700A2352
:1006F000E37110BDA401002008B5FFF7EFFF024B26
:1007000000221A7308BDC0467800002008B5054BCA
:1007100000221A70044A01231370044A1370FFF771
:10072000FBFD08BD9C01002060000020AC00002003
:1007300007B5074B022000930121064A1F2301F051
:10074000B9FE002803D10220034901F089FE07BD4C
:10075000C10A0000C40100203107000008B5FFF7FE
:10076000E7FF08BD134B70B500241C70124B134AF1
:100770001C7001231370124A1370FFF749FF114ECA
:100780003070A04201D1002511E001383070FFF730
:10079000BDFD051EF7D03378A34206D3201C0021EF
:1007A0000134FFF748FFE4B2F5E7FFF7C1FF281C6B
:1007B00070BDC0469C0100209D010020600000200B
:1007C000AC0000208401002007B5074B8120009376
:1007D0000021064A0D2301F06DFE002803D181207F
:1007E000034901F03DFE07BD5D07000078000020D1
:1007F000C907000038B5094B094C9A681D1C002A2E
:1008000006D0237B81207F2B00D8022001F09AFDA7
:1008100064686C60FFF7D8FF38BDC04678000020E0
:10082000C401002008B5064B1B78002B06D002201F
:1008300001F088FD0220034901F012FE08BDC04608
:100840009D0100202508000008B5064B1B78002BF1
:1008500006D0812001F076FD8120034901F000FEE1
:1008600008BDC0469D0100204908000010B50C1CC1
:10087000002807D1FFF740FF034B9A68141B9C60C8
:10088000FFF7B8FF10BDC0467800002008B5184B30
:1008900060211A7850B20A4000280FDA0020202A7E
:1008A00025D15A78FE2A22D1DA88012A1FD1598807
:1008B00081421CD10F499A81996017E00020202ABB
:1008C00015D15A78FF2A12D1DA8882420FD15B887B
:1008D00083420CD1084B1870084B1870022001F0AD
:1008E0008BFC812001F088FCFFF722FF012008BD6E
:1008F000CC060020840100209D0100209C010020E6
:1009000038B5051C0C1CFFF7E9FE074B01221A73D2
:10091000064B0022DA701A715A719A71220A9D7080
:100920001A735C7338BDC04678000020A401002013
:1009300008B5E82102208901FFF7E2FF08BD08B5EC
:100940000620A0218140FFF7DBFF08BD08B5042089
:100950000021FFF7D5FF08BD07B50B1C0649021C97
:1009600000918120012101F0A5FD002803D1FFF7AE
:10097000EDFFFFF73FFF07BD6D08000008B59021B0
:1009800005208901FFF7BCFF08BD000008B5094B31
:100990001B7B594049B2002904DB074B9A680123AD
:1009A000824204D2FFF7EAFFFFF724FF0023181C5E
:1009B00008BDC046C401002078000020F7B5214CD6
:1009C000071C0021201C142202F0F2FD1E4E002FF5
:1009D00004D0231CF27D0833082502E0F27C231D9D
:1009E0000425707C3F2101401C2901D03F2907D1FB
:1009F0001C2119700A2159700C350521D970EDB2EE
:100A00002B1C954200D9131CDBB2181C80210193CA
:100A1000FFF7BCFF002813D0707BFFF713FE431EC7
:100A20009841C001002F04D0023D2D022580E070C6
:100A300002E0013D2570A070201C0199FFF78CFF9A
:100A4000F7BDC04688010020C401002038B5051C50
:100A5000164C0CD1607BFFF7F5FD002807D09C21D8
:100A600007208901FFF74CFFFFF7C4FE1CE0104B85
:100A7000627C291CDA70A27C9A70E27C5A70227D1A
:100A80001A700C4BA27D5A70E27D1A7018884B1EAA
:100A900099414002C901FFF779FF002804D0064BB5
:100AA00001221D70054B1A7038BDC046C4010020DC
:100AB000A00100209E010020C00100209C01002018
:100AC000F8B5002800D0D9E01F2905D16C496D4B3D
:100AD0000A680C1C9A4207D06B4B01221A70FFF770
:100AE000A1FEFFF7B1FEC9E04A7B0F231A40674B16
:100AF0004A731B78934200D2AFE0654B8D689D60CE
:100B0000CB7B1E2B00D1A5E00DD8122B2DD004D805
:100B1000002B67D0032B18D0A5E01A2B5FD01B2B1E
:100B200000D18EE09FE02A2B00D199E006D8252B3A
:100B300064D00120282B00D192E094E02F2B00D12B
:100B400099E001205A2B4AD08DE0CB7C1C1C122B43
:100B500000D91224E4B2201C8021FFF717FF0028DF
:100B600000D18BE04B48211C68E0CB7C1D1C242B62
:100B700000D92425EDB2281C8021FFF707FF0028AB
:100B80007CD0237C990768D1677C002F65D1607B7E
:100B9000FFF760FD404E431E9841C0017070607BBE
:100BA000FFF760FD411C301C1030102202F0BEFC2B
:100BB0003B1C301CC118097CDAB2002905D022295F
:100BC00003D00133102BF5D11A1C102A05D083183D
:100BD000202101321974D2B2F7E7291C2EE0FFF769
:100BE000EDFE4BE0101CFFF715FD022823D0032873
:100BF0001ED000283FD0FFF7A9FE39E00820802151
:100C0000FFF7C4FE002839D0607B244C211CFFF77D
:100C100009FD02280FD003280AD00028EBD1226852
:100C200080239B02636013BA2360201C082105E027
:100C3000FFF785FE1CE0FFF77BFE19E0FFF78CFE57
:100C40001CE0CB7C9D0716D501219943101CFFF7B2
:100C5000F2FC10E0CB7C002B0DD0FFF78FFE07E0FD
:100C6000FFF7F4FE0AE0802105208901FFF748FE26
:100C7000FFF7C0FD02E0FFF73FFDF9E7F8BDC04612
:100C8000C4010020555342439D01002084010020EF
:100C900078000020A401002088000020B801002076
:100CA00010B51B4A00231178181C99422ED0194CFC
:100CB00013702370184B19491878194A194B0028DA
:100CC00005D0487B11681A88FFF7D4FC04E0487B04
:100CD00011681A88FFF7E0FC2378002B02D000236C
:100CE000237012E0022809D0032804D0002808D17C
:100CF000FFF702FD07E0FFF722FE04E0FFF718FE12
:100D000001E0FFF723FEFFF775FD012010BDC0468F
:100D10009C010020AC000020C0010020C401002084
:100D2000A00100209E010020F7B51A4D1E1C2B7853
:100D30000F1C141C002B01D1002029E000232B7074
:100D40000223002800D08123321E00D1124A0092D3
:100D5000181C00213A1C231C01F0ACFB002802D116
:100D600001232B7014E0002E0ED12B78002BFCD029
:100D70000A4B1A78002ADFD1094A1B7891680120B2
:100D80000C1B9460584003E0054B9A68141B9C6050
:100D9000FEBDC04660000020C1060000990400208E
:100DA0007800002008B5034B58887F23184001F0D5
:100DB00031FC08BDCC06002030B5144B1A78002356
:100DC0009A4221D0124B1B681B681A79824201D8C3
:100DD000002319E0DC789D780E4A24022C4313602E
:100DE0001C199C420ED95D78042D08D19D7885424E
:100DF00005D1DD788D4202D11360012304E01D7816
:100E00005B19EEE71360E3E7181C30BDEE0100202C
:100E1000E8010020F0010020094B1B681B68DA780C
:100E2000997812020A439B1802788018834205D9E8
:100E30004278042A02D0052AF6D100E0002070474B
:100E4000E801002038B5051CFFF7B6FF002801D1E6
:100E5000002018E00C4B1C68201CFFF7DDFF041E6F
:100E60000AD06279237912028078E1781A4301F07E
:100E700005FA0028F0D1EBE7044BAD001B685B6876
:100E8000EB581B68984738BDF0010020E8010020AE
:100E900070B50021051CFFF78FFF041E19D00E4B03
:100EA000AA001B685B68D658F3689847011C281C89
:100EB000FFF782FF041E0CD0084B1D68281CFFF7AB
:100EC000ABFF051E03D0807801F0B8F9F6E7736830
:100ED0009847201C70BDC046E8010020F0010020AA
:100EE00008B501F0F3FB08BD38B50C4B00241A78A7
:100EF0001D1CA24205D100232B70094B01221A8030
:100F000038BD084B1B681B681B79A342F3D9201C12
:100F10000134FFF7BDFFE4B2F3E7C046EE01002065
:100F2000EC010020E801002010B50B4B00241B78D9
:100F3000A3420FD0094B1B6819680A79A24209D94C
:100F40005B68A200D3581B69002B00D0984701347E
:100F5000E4B2EFE710BDC046EE010020E80100203A
:100F6000F8B5A44C0023A38123616361237858B2B0
:100F7000002803DAE288002A00D19FE160211940AD
:100F800000D051E11F22002800DBA9E0E588002DF8
:100F900000D149E1134067D16378062B09D0082BB3
:100FA0005DD0002B00D03FE1022D00D03CE1924803
:100FB00092E06088050A022D0CD006D8012D00D0E1
:100FC00032E18E4B1868017840E0032D1FD00F2DC1
:100FD00013D029E1894BC0B219684A7C824200D8FB
:100FE00022E15B68C000C058C178837809021943C8
:100FF00001F020FBA26855702AE0804B9868002819
:1010000000D111E1C1788378090219431EE0C0B212
:10101000032800D908E102F08BF9070004000A0058
:101020004E010F21764A04E0764804210EE0764A0C
:101030001621002375485D00D65C451901336E808A
:10104000DDB28D42F6D349000231017001F0F2FAAF
:10105000E388A2899A4200D8CAE0A381C8E0012DA2
:1010600000D0E1E06A4837E0012B25D163780A2BF4
:1010700000D0D9E0012D00D0D6E0654B1B78002BC5
:1010800000D1D1E0634B26791F683A681379B342E7
:1010900000D8C9E0301CFFF78FFE051E00D1C3E069
:1010A0007B68B600F358DB6898475B4B01211870EA
:1010B000181C01F0BFFA99E0022B00D0B4E063786D
:1010C000002B00D0B0E0022D00D0ADE0207901F07F
:1010D00031F9524B1880181C291C01F0ABFA87E03B
:1010E00013404CD160780138082800D99CE002F008
:1010F00015F90C9B9B9B059B9B9B1A00E388002B7F
:1011000000D091E0464B236172E0E388002B00D0D1
:101110008AE06388012B00D086E0374B02211A88D1
:101120008A431A8064E0E588002D00D07CE001F05D
:1011300079FA002800D177E0304EA27831684B7CF4
:101140009A4271DCFFF7D0FEA378314A1370002B6E
:101150004ED034492F4A5B187168DB00CB181360FE
:10116000161C33681B681B79AB4241D9281C00212F
:10117000FFF768FE002857D00135EDB2F1E7012BEB
:1011800015D163780B2B4FD1E388002B4CD1204B2A
:101190001B78002B48D025796688281CFFF778FE3D
:1011A000002841D0F1B2281CFFF74CFE1DE0022BB5
:1011B0003AD16378012B02D0032B0AD034E0E388C4
:1011C000002B31D16388002B2ED1207901F02EF92C
:1011D0000BE0E388002B27D16388002B24D12079F2
:1011E00001F00AF8207901F0ADF8051C002D1BD0A4
:1011F000012064E0CC060020EC010020B8000020B3
:101200001301002054010020FC00002024010020D4
:10121000EE010020E8010020F4010020E40100209C
:10122000A50D0000FFFFFF1F22781F231340012B95
:101230001FD1234B1B78002B1BD0224B25791E6816
:1012400032681379AB4214D9281C0021FFF7B4FD92
:1012500000280ED07368AA00D658F3689847011C7E
:10126000281CFFF7A9FD002803D0B3689847002881
:10127000BED122781F231340022B1FD1104B002414
:101280001B78002B1AD00F4B1B6819680A79A242F1
:1012900014D95B68A200D558E9688847011C201C56
:1012A000FFF78AFD002809D0AB68984700289FD136
:1012B0000134E4B2E7E70C21034ABAE60020F8BDA6
:1012C000EE010020E8010020BF3600000A4B1A683A
:1012D000002A0CD1EFF310800021084A884205D182
:1012E00072B6BFF35F8F06480170012111701A6852
:1012F00001321A607047C046F8010020FC0100204E
:1013000058010020084B1A68013A1A601B68002B2C
:1013100009D1064B1B78002B05D0054B01221A7012
:10132000BFF35F8F62B67047F8010020FC01002018
:1013300058010020002806D0034B002258609A6014
:101340001A68D103FCD5704710E000E008B5002012
:1013500000F0A4FBFA21890001F0F4FF054BFA210B
:101360001860890001F0EEFF034B05221860034B63
:101370001A6008BD600100205C01002010E000E060
:1013800010B5041C002C05D0034B013C1868FFF776
:10139000D1FFF7E710BDC04660010020024B58693D
:1013A000012318407047C0460040004138B51D4B2E
:1013B0000421DA691C4C0A43DA61A269202392B243
:1013C000FF3313432383051CFFF7E8FF031C0520AD
:1013D000002B25D0EA786B782978DB0192041A4338
:1013E000C02309029B000B401343AA781E21520020
:1013F0000A4029791343C022090492020A40134388
:101400006360A268094B5203520F08219140198072
:10141000A2685A806A781A71A069C005C00F0001DD
:1014200038BDC0460004004000400041FE010020DD
:10143000F8B51F4B041C5A881B880E1C5A431823EE
:10144000914233D81B4D80236F68DB023B436B60B6
:10145000AA69202392B2FF3313432B83FFF79EFF29
:101460000523002822D0062C06D89C420BD2022C41
:101470000DD0042C19D10AE0402C16D3412C06D9EA
:10148000452C07D911E0AA691023D1050ED4B6085E
:101490007600EE61A5231B021C432C80FFF77EFF24
:1014A0000028FBD06F60002300E01723181CF8BD54
:1014B000FE01002000400041F8B5214B0E1C151C18
:1014C00059881A88041C51431823884235D8511E64
:1014D000014232D1172395422FD8FFF75FFF052332
:1014E00000282AD0174F184B3B80FFF757FF0028E2
:1014F000FBD0BA69202392B2FF33134360083B83C9
:10150000400000239AB2AA420ED29AB26F1EB15C7A
:10151000BA4201DB0A1C03E0B218527812020A43F5
:1015200019180A800233EDE700233F2D05D81A1C55
:101530000420211CFFF77CFF031C181CF8BDC046CB
:10154000FE0100200040004144A5FFFFF8B5194B03
:101550000E1C19885B88141C4B43051C18229842EA
:1015600025D84F1E074022D117228C421FD8FFF7E3
:1015700015FF052200281AD00F4B20229969FF324F
:1015800089B20A436D081A836D003B1C9AB2A242CD
:101590000CD25A191188601E89B29AB2B154824293
:1015A00002DAB218090A51700233EFE70022101C68
:1015B000F8BDC046FE0100200040004138B5104B88
:1015C000041C1D885A8818236A43904215D8AD0020
:1015D000013D054011D1FFF7E1FE052300280CD0A5
:1015E000084B20229969FF3289B20A431A83A40862
:1015F000054A6400DC611A802B1C181C38BDC046EB
:10160000FE0100200040004102A5FFFF024B1868C8
:101610000004C00F7047C0460018004008B5054BD5
:1016200002211A68D2B20A431A70FFF7EFFF0028AE
:10163000FBD108BD0018004007B5124B40219A6944
:1016400005200A439A6101A900230B7000F09CFA5F
:10165000052000F05DFA0C4B01211A68D2B20A4352
:101660001A70FFF7D3FF0028FBD1084B0022C318E4
:1016700004301A604028F8D1054B10221A60FFF799
:10168000CDFF07BD00040040001800409C0400206E
:1016900000E100E010B50B4C0023237023780F2BE2
:1016A0000FD8094A012110699940084206D01161FA
:1016B000064A9B009B58002B00D0984723780133A3
:1016C000EBE710BDDC040020001800409C04002063
:1016D00007B5802201AB1A700A785A704A789A705E
:1016E0008A78191CDA7000F0B1FA07BD10B50C4BFE
:1016F00002211A680A431A60196880229143094A34
:1017000089B29184101CC168064ACC06FBD5996841
:101710000020D162596891621B689BB2938410BD0E
:10172000040200200008004010B5082832D801F05B
:10173000F5FD0831310505130B1629008020000244
:101740002BE0164B186928E0154B186A154B8005DD
:10175000800FC340181C20E0104B58691DE00F4C4F
:1017600002232068184018D00D4BDB68DA06FBD541
:1017700023685A0710D5002000F012FAA3689BB224
:1017800058430AE0064B00201B6D5A0705D5034B52
:10179000D86802E0002000E0034810BD04020020E9
:1017A0000008004000127A00006CDC0270B50D4B9E
:1017B00045781E6A817804780122402086431540CE
:1017C000AD01301C0A402843D10180229043021C05
:1017D0000A43054803212140090202400A431A62D4
:1017E00070BDC04600080040FFFCFFFF30B5027A24
:1017F000438992069B059B0D120C1A43124B81885C
:101800005A604288C4791143827922430A4341785D
:10181000C9010A431A600278042A0BD1047BC189EA
:10182000058A0A48A40609042C4301402143996013
:10183000196806E0202A06D1028A9A601968842273
:10184000D2000A431A6030BD040200200000FF03EA
:1018500008B508282CD801F061FD122B2B100B19AC
:1018600005202300134B02211A6A0A431A6204E07E
:10187000104B02219A690A439A61002019E00D4B2E
:1018800002211A6992B20A431A82F6E7094B022131
:101890005A6992B20A439A82EFE7FFF727FF08E0FE
:1018A000044B5A6C0223D2B21A43034B1A70E4E77A
:1018B000172008BD000800404408004010B5C223AE
:1018C0002D4CDB00A3602D4B1E215A688AB08A4341
:1018D00004210A435A6005A80023438083714370A2
:1018E000072303733F232022C381254B02701A680C
:1018F000920E3F2A00D11F22224B23491B689B05D1
:101900009B0D8B4200D1214B43810823C37180235F
:101910005B0083801E4B02720382FFF767FF01A802
:1019200000230122437082700370FFF73FFF0620FF
:10193000FFF78EFF00F038F8FFF7D8FEE2680E4B95
:10194000D106FBD59A8C80210A439A84114B00243E
:101950001C7202A95C7207229C72201C01234B603E
:101960004C704C720A700B7200F02EF8201C00F0C4
:1019700079F80AB010BDC0460008004000400041A0
:101980002460800028608000FF030000FF01000049
:1019900080BBFFFF00040040024B18680004C00F2A
:1019A0007047C046000C0040054B08219A690A4365
:1019B0009A61044B01221A701A68D107FCD470474F
:1019C00000040040000C004070B50C784B782402F5
:1019D000051C061C0443002B02D08023DB021C43A1
:1019E0004B7A002B02D080231B031C434B68012B36
:1019F00013D95E1E1E400222002E09D19A4202D245
:101A000001365200FAE7360280232E435B0303E0DF
:101A10001E0280232E439B021C430B7A002B02D014
:101A200080239B031C43FFF7B7FF0028FBD1FFF780
:101A30004DFC0A4B1D70FFF7AFFF0028FBD1084D8E
:101A4000AE60FFF7A9FF0028FBD16A6880235B0224
:101A500013401C436C60FFF755FC70BD080C004040
:101A6000000C004010B5041CFFF796FF0028FBD1C6
:101A7000FFF72CFC074B1C70FFF78EFF0028FBD1F3
:101A8000054B8022596852020A435A60FFF73AFC1C
:101A900010BDC046040C0040000C0040F8B5071C07
:101AA000FFF77AFF0028FBD1FFF710FC154B1F70E2
:101AB0001E1CFFF771FF0028FBD1134D6868C0049E
:101AC000C00EFFF731FE37706E68104BF602041C33
:101AD000F60F1F70FFF760FF0028FBD1AD682D02E5
:101AE0002D0CFFF70FFC002E07D1012D07D9201C6C
:101AF000291C01F027FC041C01E00135EC40201CEE
:101B0000F8BDC046040C0040000C0040080C00402A
:101B100010B5041CFFF7DAFB054B80221C70054B47
:101B2000D2011968090C0A435A80FFF7EBFB10BD7C
:101B3000020C0040000C004038B5041CFFF7C6FB47
:101B40000D4B0E4A1C700E4B0E4C1968588809013B
:101B5000104058801868090F000C20405880101C55
:101B60001C68074A6500FBD45388090203400B43F5
:101B70005380FFF7C7FB38BD020C0040FFF0FFFFAA
:101B8000000C0040FFBFFFFF10B50C782402044397
:101B9000FFF7D2FF014BA4B25C8010BD000C0040E7
:101BA00010B5041CFFF792FB054B1C70054B1C681D
:101BB000FFF7A8FB2401240F201CFFF76FFF10BDC7
:101BC000020C0040000C004030B5D47800239C4249
:101BD0001BD11478802C03D0802324065B0223437E
:101BE00054780225AC4309D19478002C02D180248A
:101BF000A40201E0C024E402234341605478013C84
:101C0000E4B2012C01D8104C2340A0248DB2E4058D
:101C10002C431C438462D0240D0C24062C431C430B
:101C20008462D478002C0DD15C0305D59378012B08
:101C300001D1816100E041615378013BDBB2012BAE
:101C400000D8816030BDC046FFFFFBFF08B5031C14
:101C50000A1C4009D90903D10549C001401800E018
:101C600000201F210B4001219940FFF7ADFF08BD67
:101C700000440041704708B5FFF720FEFEF7B0FCB6
:101C8000FFF7F8FFFFF7D8FC08BD000008B5044BCC
:101C900001229A71034B1B68002B00D0984708BDA6
:101CA00000100040E0040020EFF3108072B6BFF394
:101CB0005F8F034B00221A70434258417047C04661
:101CC000580100200F2303405B00C0091818023898
:101CD00014235843014B18187047C04620020020B7
:101CE000F0B58E7985B073B20D1C0F27301C002B18
:101CF00046DAFFF7E7FF6D88C368028AED1883684C
:101D000037400197041C0292C560877C9D4221D018
:101D10005E1B4B4AB6B2964206D9101C029901F0DE
:101D2000B5FB474B5E1AB6B20023BA0706D5301C86
:101D3000029901F04BFB8BB25A4253415A00A37CEB
:101D400002218B4313436268A37452193D480199E1
:101D5000331C0AE0B807C00F0AD0022362689F4311
:101D600038480199A7745219002300F0F3FE64E08B
:101D700001239F432368A774002B5ED0291C5AE0DF
:101D8000FFF7A0FF038A37400193837C0297041C6E
:101D90002F885A0710D5C268436801999B1880683C
:101DA000039301F013FB0A1C0299274B01398901A7
:101DB000C918039801F0BAFBE368FA18A368E26057
:101DC0009A4200D9E360AA88BA422BD1E5689D42C5
:101DD00028D05E1B1A4FB6B2BE4206D9381C0199F4
:101DE00001F054FB7F1ABBB206E0301C019901F0F0
:101DF000EDFA8BB2F61AB3B2019A124893420BD2A3
:101E0000A37C04221343029AA374013A0E4B92015D
:101E1000D2180299019B02E062680299521900F0FF
:101E2000BFFE0AE0A37C01229343A3742368002B26
:101E300003D0E1680020321C984705B0F0BDC046D1
:101E4000FF1F000064050020E404002010B5064CCC
:101E5000064B0522201C80211A7000F03DFE201C3C
:101E6000002100F046FE10BD640500207402002031
:101E700037B5041CFFF738F8226801AD8023937250
:101E8000281C00F027FD0323291C201C6B7000F088
:101E900029FD201C174900F0A7FE201C002102226A
:101EA000154B00F063FC00210A1C201C134B00F0B2
:101EB0005DFC134B201C0021012200F057FC201C6C
:101EC0000021022200F07AFC00210A1C201C00F0F4
:101ED00075FC201C0021012200F070FC2368094AD7
:101EE00019890A408021C9000A431A81064B002241
:101EF0001A7037BDE406002041200000692300006D
:101F0000411F0000FFF3FFFF7402002010B5084CD2
:101F1000084B0322201C08491A7000F065FE074B8D
:101F200000219A68201C0B1C00F014FE10BDC04656
:101F30006405002074020020E4060020CC06002086
:101F400008B589790C4B4AB2002A08DA1B78012BB4
:101F500002D1FFF7DBFF0DE0042B0BD107E01A786D
:101F6000022A02D104221A7004E0032A02D1034893
:101F700000F0B2FD08BDC0467402002064050020D8
:101F8000F8B51D4D1D4E2B88B4891D4FE41AA4B21F
:101F9000002C1BD11B4A11885B189BB21380F2885E
:101FA0009A4203D0184B1B78002B07D0174B042202
:101FB000381C17491A7000F017FE1CE07369002BDB
:101FC0000BD09847002808D02C80B4893F2C04D926
:101FD0000D4B00221A70402402E00B4B01221A70B4
:101FE0002B88B268381CD2180021231C00F0B2FDE7
:101FF0002B88E4182C80F8BD70020020CC0600204D
:10200000640500201C0200207202002074020020DF
:10201000E406002008B5FEF787FFFEF76BF908BD60
:10202000064B5A6A910605D4D968D0220A40D02AB4
:10203000FAD102E0DA68D106FCD57047000800400A
:1020400070B5284E0C1C3378002B06D0264B1B692C
:10205000002B00D09847002333702388082B02D030
:10206000FFF7F4FE3CE0214C1F4D2378A2782B7043
:1020700063786B70E3781B02D3186B8063792279E5
:102080001B02D318AB80E379A2791B02D318EB8033
:10209000FEF766FF0028E3D02B787F2B0ED9144B78
:1020A00000211980134B221C19800223337012481F
:1020B000402300F075FDFFF763FF11E0EB88002B74
:1020C00002D1FFF723FF0BE0094B00211980094BD8
:1020D0000948198001233370221C402300F060FD61
:1020E00070BDC04674020020CC060020E40600202B
:1020F0001C0200207002002064050020002805D08A
:10210000034B01221A70BFF35F8F62B67047C0465F
:1021100058010020F7B501AE041C1149301C0422FF
:1021200001F004FA0F4B1D78A54217D0002C08D0FF
:10213000375DFFF7B9FD0C4BDA5D0132DA55FFF779
:10214000DDFF002D08D0755DFFF7AEFD064B5A5D33
:10215000013A5A55FFF7D2FF024B1C70F7BDC0463B
:10216000CC360000730200209404002010B5084C07
:102170000621201C00F0ECFA201C042100F0E8FAF3
:102180000221201C00F0D4FA0220FFF7C3FF10BD8B
:102190006405002010B5FFF743FF0C4C0221201C02
:1021A00000F0D6FA201C042100F0C2FA084A201CD4
:1021B000062100F0ADFA0621201C00F0B9FA032038
:1021C000FFF7A8FFFEF792F810BDC0466405002097
:1021D0006D21000010B5074C0421201C00F0B8FA56
:1021E0000221201C00F0A4FA0120FFF793FFFEF764
:1021F00079F810BD6405002038B5041C211C0A487C
:1022000000F045FC201CFFF75DFD827C031CD1071C
:1022100008D501201D6882439A74002D02D0D96828
:10222000221CA84738BDC04664050020024B1B682D
:1022300018698004400D704764050020F7B501ADB2
:10224000041C281C00F046FB201CFFF7D5FF0A4F9A
:102250000026291C381CEE702C7000F043FB0F2167
:10226000321C2140381C00F095FA381C321C211C0D
:1022700000F0EAFAF7BDC04664050020F7B501ACEE
:10228000061C201C0F1C151C00F024FB26700023CC
:10229000082D1DD90123102D1AD90223202D17D95D
:1022A0000323402D14D90423802D11D980235B00F2
:1022B0009D4201D805230BE080239B009D4201D85D
:1022C000062305E0184B9D4201D900202BE007238F
:1022D000301C6370FFF7F6FC0323391C058219409C
:1022E000012901D1022304E0022902D00329ECD103
:1022F00004230E4D211C281CE37000F0F3FA041E89
:10230000E3D10F210A4B3140221C281C00F02EFA89
:10231000311C221C281C00F051FA281C311C0122FF
:1023200000F04CFA0120FEBDFF0300006405002010
:10233000E11C000008B5011C014800F0BEFB08BD0F
:10234000640500200F2310B50340041C0020022B5D
:1023500007D80448211C00F0BFFB201CFFF74CFFEE
:10236000012010BD64050020F8B52A4E3378012BFA
:1023700043D1294A294C0D881788A38979198B42A2
:1023800001DADD1BADB2A2682549D0192A1C01F083
:10239000CDF8EF19204ABBB21380214F402D05D153
:1023A000204DE1882A88D218914209DCA381636913
:1023B000002B02D0984700280BD0FFF7A7FD28E09C
:1023C000A2899A4212D16069002802D08047002871
:1023D00004D105233370FFF7B5FF1AE00E4B1A88BE
:1023E0002B88D3180C4A2B800023138000213A1C21
:1023F00040230D4800F0D4FB0BE0022B02D1FFF785
:10240000BFFD06E0054B1B69002B00D09847002359
:102410003370F8BD7402002070020020CC0600204A
:10242000E40600201C020020640500200F2370B584
:102430000340061C0024022B0ED8FFF743FC311C7E
:10244000051C064800F055FBAB7C0124DA0703D5D8
:10245000A343AB742B689847201C70BD6405002013
:10246000F7B50F23051C01910340022B01D900246D
:102470001BE0FFF727FC837C061CDA07F7D40C4F20
:10248000291C381C00F019FB041E06D0B37C012265
:102490001343B374019B336007E0381C291C00F020
:1024A000E5FA041EE3D0019A9047201CFEBDC04609
:1024B00064050020F0B51E1C0F2385B00340071CE7
:1024C000029103920193022B01D9002597E0FFF7B7
:1024D00031FF051EF9D1381CFFF7F4FB041CFFF790
:1024E000E3FBA27CD10702D5FFF708FE87E00123BA
:1024F0001A43A274002804D0424A1370BFF35F8FBE
:1025000062B60023E3600A9B039A0298A17C2360D1
:102510000123626018400222984091430143042045
:102520008143A17479B2A660002930DA002E1AD056
:10253000354DB6B2AE4205D9218A281C00F0A6FF5F
:102540006E1AB6B202990023994206D0218A301C35
:1025500000F03CFF8BB25A4253415A00A37C022147
:102560008B43134304E00299002909D0A37C9343D1
:10257000A3740199039A331C244800F0EBFA3BE062
:10258000A27C9A43A2740A9A002A08D10CE0002E79
:102590000CD1A27C0A999A43A274002904D000208D
:1025A000011C3A1C0A9B9847012528E0164FB6B239
:1025B000258ABE4206D9381C291C00F067FF7F1A05
:1025C000BBB206E0301C291C00F000FF8BB2F61AEB
:1025D000B3B20E48AB420BD2A37C04221343019A40
:1025E000A374013A0A4B9201D21801992B1C01E005
:1025F0000199039A00F0D4FA45424541EDB2281CF6
:1026000005B0F0BD58010020FF1F00006405002048
:10261000E4040020024B80221B681043987270472C
:1026200064050020024B1B6898684002400E70470A
:1026300064050020014B986099817047CC0600200A
:1026400038B50320FFF766FD1A4C01252368201CCE
:102650009A68042192B2AA431A81174A00F058F8E6
:10266000201C0021154A00F053F8291C201C144A94
:1026700000F04EF8134A201C022100F049F8201CFB
:10268000042100F055F8201C002100F051F8291C0D
:10269000201C00F04DF8201C022100F049F80A4AE5
:1026A000201C062100F034F8201C062100F040F820
:1026B00038BDC04664050020D5210000152000006B
:1026C000711E0000952100006D21000073B5FFF719
:1026D000EBFA01AC061C201C00F006FD0A4D00239D
:1026E0000A49221C281CA37000F006FD281C00F0DB
:1026F00093FAFFF795FC0120FFF70CFDFFF7A0FF11
:10270000301CFFF7FBFC73BD640500200050004146
:102710000B1C2E339B001A50044AAA235B0049006D
:10272000895AC25A0A43C25200207047D03600006C
:10273000064B49000268CB5A9383AB225200815A60
:10274000194381520268002013837047D03600007D
:10275000054BAB2252004900CB5A815A9943815212
:102760000268002093827047D036000010B58C00BC
:10277000A4183434A4000419411863605931044B7F
:10278000FF3108789B5C03430B70002010BDC046EE
:10279000DE36000010B58C00A418031C34345B181E
:1027A000A40004190449002059336060FF33895C98
:1027B0001A788A431A7010BDDE36000070B50F23F8
:1027C0000B40C41861341F4DFF342678AD5C35438F
:1027D0002570002A0ED10268002B02D1FF3203239C
:1027E0000FE05B01D31849B2FF330222002926DB38
:1027F000012224E0012A0FD10268002B03D1FF320D
:102800000C2393721CE05B01D31849B2FF330822FA
:10281000002914DB042212E0022A05D102685B01C0
:10282000D318FF3310220AE0032A09D102685B01A2
:10283000D31849B2FF334022002900DB20229A72CC
:10284000002070BDDE36000070B50F230B40C418A9
:102850001F4D6134FF34AE5C2578B5432570002AE6
:102860000ED10268002B02D1FF3203230FE05B017F
:10287000D31849B2FF330222002926DB012224E0CB
:10288000012A0FD10268002B03D1FF320C235372AF
:102890001CE05B01D31849B2FF330822002914DB86
:1028A000042212E0022A05D102685B01D318FF332B
:1028B00010220AE0032A09D102685B01D31849B249
:1028C000FF334022002900DB20225A72002070BD15
:1028D000DE36000000230370437083700123C37051
:1028E00070470000F0B5021C0D78C8780F232B400C
:1028F000ED09042800D998E0146800F00FFD0308E2
:10290000495D7A0008335B010020E054A9E05D01D5
:102910006419FF3466781C20770700D0A1E067783F
:102920007026374200D09CE0112060701468083394
:102930005B01E018402444711268D31880221A7198
:102940008A78484B002A08D05A195468802000061B
:10295000044354605469204307E05A19506840000A
:102960004008506050694000400850615D194C7843
:10297000686807223C4B14401840240720436860D5
:1029800049780A40696912070B4013436B6162E0A2
:1029900058012418FF34002D07D0677870261C20BA
:1029A00037425ED16078202612E066781C207707D7
:1029B00057D1607802262FE058012418FF34002DEB
:1029C00010D0677870261C2037424AD160783026B4
:1029D0003043607010681A1C08325201821880203F
:1029E000107122E066781C2077073AD160780326C0
:1029F00012E058012418FF34002D07D067787026A4
:102A00001C2037422DD160784026E1E766781C20F3
:102A1000770726D1607804263043607010681A1C4E
:102A2000083252018218402050715B005D190D4B35
:102A300048782D015B19072210405C680A4A00079C
:102A4000224002435A608878002806D059688022C4
:102A500012060A435A60002003E05A6852005208E6
:102A60005A60F0BD24070020FFFFFF8F0F220A40AD
:102A700003680832520149B29858002901DA400629
:102A800000E04007400F431E9841C0B270470F233B
:102A90000B40026808335B0149B2D218002905DAFD
:102AA000802111710268D318022204E04021517183
:102AB0000268D3180122DA7170470F220A400368B6
:102AC000083252019B1849B25868002901DA800285
:102AD00000E0C002C00F70470F220A4003680832AE
:102AE000520149B29B182022002900DB10225A71A2
:102AF000704730B50F220A404CB201685301C91823
:102B0000FF31CD79002C11DA2024254220D04C71E0
:102B10000168CB18FF331C7A40210C4218D019727F
:102B20000368083252019A18022310E0102425424B
:102B30000ED04C710168CB18FF331C7A20210C4257
:102B400006D019720368083252019A1801231371D2
:102B500030BD000070B50D1C046808356D012E599C
:102B60001C247606760F14D00B4C490161180A61BB
:102B70000C1C0A4A49690A4062619A046369920C12
:102B80009B0B9B0313436361036800245D1980233F
:102B90006B71201C70BDC04624070020FF3F00F071
:102BA00070B50D1C046808356D012E591C2476077C
:102BB00013D00B4C49010A5161184C689A04094B17
:102BC0001209234013434B604B6800249B0B9B036B
:102BD0004B6003685D1940232B71201C70BDC046FB
:102BE00024070020FF3F00F0094B0A4A196059688A
:102BF0000A40802189020A435A605A68920B920364
:102C00005A6003684022FF3300205A717047C04663
:102C100024070020FF3F00F0036802211A68D2B2A7
:102C20000A431A70026813681B021B0E022BFAD0AB
:102C300070470000F0B5D04E85B0346825682B6829
:102C40001B06DB0F00D13FE1286A80B200F02AFCAE
:102C5000071E1F2F00D9BDE0021C08325201AD181B
:102C60006D6803202D0E054242D0C448012103683F
:102C7000B9408B430360216803238818E119C371AD
:102C8000A83189790120014232D0BD4B1F702168E3
:102C90005058BC497A0180078A18800F5168012872
:102CA0000BD18904890C598051680901890C9980DC
:102CB00053689B0B9B03536013E00901890C88B296
:102CC000029059805168B0488904890C99805168F4
:102CD000084050600298002803D152689204920C78
:102CE0005A80BB1C1B01E3185B68201CA449984751
:102CF00004231D420CD0A14A01211068B940884329
:102D00001060326811683A1C083252018A18D37177
:102D100008231D421ED0994A01211068B9408843FA
:102D200010603068FA18016852018A18D371C3190B
:102D3000A8339B799A070DD5924A91497B01D31804
:102D40000F7008335B68DB02DB0E4B703B01C3186E
:102D50009B6A984710231D421FD0884A01211068A2
:102D6000B9408843106030683A1C0168083252014B
:102D70008A18D371C319A8339B795A070DD5804B94
:102D800080497A011F708A18526800211201920C42
:102D90005A803B01C318DB6A984720231D4200D1AB
:102DA0009BE1764A01211568B94030688D43156072
:102DB0003A1C066808325201B218D371C319A833FD
:102DC0009B79190700D488E16D490F703F01C7193D
:102DD0003B6B81E1EF690423BFB21F4208D0AB8394
:102DE000231CA5331B78DA0702D56368201C98479B
:102DF00008231F420CD0614A306800211160056829
:102E0000AB83031CA5331B78990701D583689847CA
:102E100040231F4209D0306802689383031CA53306
:102E20001B78DD0601D54369984720231F4209D04E
:102E3000306801688B83031CA5331B781A0701D502
:102E40000369984710231F4209D030680568AB8397
:102E5000031CA5331B78590701D5C3689847802305
:102E60001F420CD0454A30680021116002689383EC
:102E7000031CA5331B789D0601D5836998478023E1
:102E80005B001F420CD03D4A002130681160016890
:102E90008B83031CA5331B785A0601D5C369984759
:102EA00080239B001F4200D117E1344A3068002183
:102EB00011600568AB83031CA5331B787F2B00D8FA
:102EC0000BE1036A984708E12A6A92B20292002A4B
:102ED0004BD1AB23ED695B00AA22E35A5200ADB29D
:102EE000A45A2B40029F1C40284B7A00D35A1D4203
:102EF00002D03268126893831C420FD02449062FF7
:102F000006D1204B9A68802312095B0013400B60A6
:102F10003B1C30682E339B001B5898470137072F06
:102F2000E2D1DAE01F1C0837B02000977901400099
:102F3000E7183E1859374919FF3730783F788C46E3
:102F400049680190090E384060270840394221D174
:102F50001027394239D10C2739424AD18E0700D087
:102F60008DE00133082B00D1B7E002990126194109
:102F7000DAB23142F5D0D5E7900200208402002079
:102F80007C02002024070020FF3F00F0D036000024
:102F90007802002059016D18FF352E7A40210E422B
:102FA00004D02972802149420A4304E02E7A20216C
:102FB0000E4202D029724A498A716022104200D121
:102FC0008BE01B01E318E03357E06146CF713278A4
:102FD0003A4200D181E043495A018A1852681B01E4
:102FE00092043F49E318920CDC330A801B68201CD2
:102FF00072E059016D18FF352E7A08273E4220D025
:103000002F72384D69188F6918256D18BE0305D5C4
:10301000896902270902090EB943A9708021494232
:103020000A432F49009F8A7121687E018E197268B8
:10303000950152D40C2210424FD01B01E318D83313
:103040001BE02E7A04273E42F4D02F72254D6918DA
:103050008F6808256D18BE0305D589680227090207
:10306000090EB943A9701E49009F8A7121687E012B
:103070008E197268D501DDD52FE01B682AE05E014C
:10308000AD19FF352F7A02210F420CD0297280250D
:1030900013496D422A438A71124A96197269920441
:1030A000920C4A8010E0297A012739420CD00C4951
:1030B0002F728A710B4A961972689204920C0A80D8
:1030C00072681201920C8A80810706D00D331B01B1
:1030D000E3185B680249201C984705B0F0BDC04664
:1030E0008802002024070020002201230270437080
:1030F0008270C37070470000F0B585B00192654AD8
:1031000000231360644A051C1060644A29600C1C8B
:10311000D169202003AE01430120D1610627B070A0
:10312000311C18207370F3703770FEF78FFD192073
:10313000311C3770FEF78AFD01996A468B78381C7E
:1031400002A91372FEF720FD381CFEF7E1FC23787C
:103150000120034323702368D903FCD450490B6832
:103160005A0B1F231A409A4200D105221A4090019F
:10317000268D4C4A3240024322850868820C134057
:103180001F2B00D11D23208D1F221340904303438A
:1031900023850B680722DB0D1340934200D10323E4
:1031A0001340218D1A03404B40480B4013432385A5
:1031B00001997F230A782178D2010B401343019AA9
:1031C0002370517801231940237804228900934306
:1031D0000B43019923706062CB78012B04D12B68DB
:1031E0000C211A898A4306E0002B05D12B680C2498
:1031F0001989A1430A431A8180220021520000F05C
:10320000D7F90023E918002204334A60202BF9D1B2
:10321000A918002310324B628B62CB620B63802AA9
:10322000F6D12A1CA43213705370E918081C00222E
:10323000A630AE31013302700A70082BF5D1131C91
:10324000E918B831002204330A601C2BF8D1A91800
:10325000081C0023D430E0311032036043608360E7
:103260000B60802AF3D1AA225200AB52AB2252004B
:10327000AB52AC20EA184000111861320020FF3236
:10328000013308701070082BF3D1094B80221A60AB
:1032900005B0F0BD84020020900200200004004030
:1032A000246080003FF8FFFFFF8FFFFF240700200E
:1032B00000E100E0FEE700001148124910B5884225
:1032C00001D0002301E0104B07E0104CCA18A242C5
:1032D000F9D2C45804331460F7E70D4A191D043BB2
:1032E000934203D200221A600B1CF6E7094A0A4BEC
:1032F0007F218A439A6000F0F5F8FCF7B5FFFEE7FE
:103300000437000000000020680100206401002054
:10331000240800200000000000ED00E002B4714627
:1033200049084900095C49008E4402BC7047C04608
:1033300003B47146490840004900095A49008E44C7
:1033400003BC7047002934D00123002210B4884206
:103350002CD301242407A14204D2814202D20901C4
:103360001B01F8E7E400A14204D2814202D24900E5
:103370005B00F8E7884201D3401A1A434C08A04288
:1033800002D3001B5C0822438C08A04202D3001B1E
:103390009C082243CC08A04202D3001BDC08224335
:1033A000002803D01B0901D00909E3E7101C10BC59
:1033B0007047002801D00020C04307B4024802A192
:1033C0004018029003BDC046D90000000029F0D08B
:1033D00003B5FFF7B9FF0EBC4243891A1847C04630
:1033E000002941D010B4041C4C40A4460123002203
:1033F000002900D54942002800D5404288422CD3FC
:1034000001242407A14204D2814202D209011B01F6
:10341000F8E7E400A14204D2814202D249005B00F5
:10342000F8E7884201D3401A1A434C08A04202D35D
:10343000001B5C0822438C08A04202D3001B9C089E
:103440002243CC08A04202D3001BDC082243002800
:1034500003D01B0901D00909E3E7101C6446002CC6
:1034600000D5404210BC7047002806D003DB002086
:10347000C043400801E08020000607B4024802A1D2
:103480004018029003BDC046190000000029EBD08F
:1034900003B5FFF7A7FF0EBC4243891A1847C04681
:1034A0007047C046414208401C2101231B0498423A
:1034B00001D3000C10391B0A984201D3000A0839C5
:1034C0001B09984201D30009043902A2105C401A7A
:1034D0007047C0461B1C1D1D1E1E1E1E1F1F1F1FCA
:1034E0001F1F1F1F70B50D4E0D4D0024AD1BAD10DD
:1034F00005D0A300F35801349847A542F9D100F054
:10350000F1F8084E084D0024AD1BAD1005D0A30006
:10351000F35801349847A542F9D170BDF036000048
:10352000F0360000F0360000F4360000F0B50F2A47
:1035300035D9031C0B439C0735D1161C103E3609A8
:103540003501451910350C1C031C27681F6067687E
:103550005F60A7689F60E7681034DF601033AB429C
:10356000F3D1731C1B01C518C9180F231340032B7B
:103570001BD91C1FA4080134A4000023CE58EE5010
:103580000433A342FAD1ED18C91803231A4005D019
:103590000023CC5CEC5401339342FAD1F0BD051CFE
:1035A000002AF5D1FAE7051CF2E71A1CF8E7C04635
:1035B000F0B54F464646C0B483B0830752D0541E80
:1035C000002A4AD0CEB2031C032503E0621E002C61
:1035D00043D0141C01335A1E16702B42F6D1032C13
:1035E00033D9FF250D402A0215432A0415430F2C19
:1035F0001AD9271C103F3F09B9463F01B84610278A
:10360000FF18BC4646461A1C664415605560956016
:10361000D5601032B242F8D14F4601373F010F2238
:10362000DB191440032C10D9271F1E1DBF0801965B
:10363000BE00B446019E1A1C664420C2B242FCD1B0
:103640000137BF000322DB191440002C05D0C9B29A
:103650001C1919700133A342FBD103B00CBC904676
:103660009946F0BD031C141CB9E7C046EB3C906DB5
:103670006B646F736673000002040100021000E4C3
:1036800001F80100E401E00100000000000000007A
:10369000000029785634124D542D44323145204DC6
:1036A00053444641543132202020224D542D44327F
:1036B000314520426F6F746C6F6164657222003710
:1036C00034383635313139353833300000030201B2
:1036D0000400080070008000010000010002030CDB
:1036E00010600000F8B5C046F8BC08BC9E467047A4
:1036F00031010000F8B5C046F8BC08BC9E467047D2
:0437000005010000BF
:103704004D542D44323145204D53440800000000EF
:1037140000000000000000000000000000000000A5
:103724004146004C004100530048000F00262E0083
:10373400420049004E0000000000000000000000AC
:10374400464C41534820202042494E0000000000CE
:1037540000000000000020084E12020000C0030018
:1037640001000000650700000D0700008D0800003F
:10377400BD06000000000000555342530000000045
:103784000000000000000000000003021F00000011
:103794004D415454414952200000000000000000F3
:1037A4000000000000000000312E30300100000055
:1037B400DC000020C4000020C8000020B00000206D
:1037C400000000006400002012010002000000401C
:1037D400D0160C0A000101020301000009022000B6
:1037E400010100C032090400000208065000070568
:1037F4008102400000070502024000004D542D44A0
:10380400323145204D534420426F6F746C6F6164B4
:103814006572004D61747461697254656368204C0B
:103824004C43000000030000000000000000000002
:103834000000000000000000000000000000000084
:103844000000000000000000000000000000000074
:103854000000000004030904010000000800000047
:04386400401F000001
:04000003000032B90E
:00000001FF
